:020000040000FA
:0400000006303A2864
:08000800A000030EA100831209
:1000100005191028831601178312B23081002B288E
:1000200083160113831203140B190310A80DA90DD5
:10003000AA0DAB0DAC0DAC16FF302C02031D2B2806
:10004000FA302B02031D2B2831152A08AF0029088E
:10005000AE002808AD008B100B11210E8300A00EFE
:04006000200E090065
:0C007400203084008001840A6030040207
:10008000031C3C281230B00085218316FF2390000A
:10009000831283160C308505870183128501870141
:1000A000073099000030831691009F008312C830FA
:1000B00083168100831231309000003083168C004B
:1000C000831210308B00DD2181018E018F010B1115
:1000D0008B100B108C018B177B2031197E20B30BFA
:1000E0007928031085190314B90DF030390203196A
:1000F000FA20F6216C28640032100800311101301A
:10010000B7008B132030370783169B001C141A0886
:100110008312A4001030370783169B001C141A08A2
:100120008312A300A6000230A6060030370783160C
:100130009B001C141A088312A200A7000130A70616
:100140008B17321CA92822090339A200A309A4098C
:10015000A50924082F02031DF42823082E02031DDD
:10016000F42822082D02031DF42801303702031D54
:10017000BE283D18BE283D143E149321023037029C
:10018000031DC728BD18C728BD143E149A2103308B
:100190003702031DD0283D19D0283D153E14A1215A
:1001A00004303702031DD928BD19D928BD153E14C6
:1001B000A82105303702031DE2283D1AE2283D162A
:1001C0003E14AF2106303702031DEB28BD1AEB2881
:1001D000BD163E14B62107303702031DF4283D1B1F
:1001E000F4283D173E14BD21B70A08303702031822
:1001F000080081280130B600B300B400B500B70094
:1002000085018701B1137B20B30B382903108519B1
:100210000314B90DF030390203195F29B40B3829E2
:10022000013037020319C521023037020319C821F2
:10023000033037020319CB21043037020319CE21D2
:10024000053037020319D121063037020319D421B2
:10025000073037020319D7219630B4000330370234
:1002600032300319B4000430370232300319B400BD
:10027000311D03293111321C42292D090339AD00EA
:10028000AE09AF092F1C03298E018F010C1C032915
:100290000C102E1E03298B1320303707BB002F08AC
:1002A000BA00722110303707BB002E08BA00722145
:1002B00000303707BB002D08BA0072218B1785016B
:1002C0008701B70AB60108303702031C0329DD2174
:1002D00008003E1C08003E101030BB003D08BA006C
:1002E000722108008B133A0883161C159A003B08EC
:1002F0009B0055309D00AA309D009C1464009C1802
:100300007E291C1183128B170800831610309B0066
:100310001C141A088312BD00FF30D000D415D51567
:10032000D615D7150800BD103D11BD110230CE0005
:10033000D20008003D103D11BD110130CE00D200A9
:1003400008003D10BD10BD118230CE00D200080063
:100350003D10BD103D114130CE00D2000800BD124D
:100360003D13BD130030CF00D30008003D123D13F4
:10037000BD130230CF00D30008003D12BD12BD13E3
:100380000130CF00D30008000800013085060800C6
:100390000230850608000130850608000230850617
:1003A000080030308506080010308506080020302F
:1003B000850608002230850608006400B30BDD299D
:1003C000B40BDD293D189321BD189A213D19A121B7
:1003D000BD19A8213D1AAF21BD1AB6213D1BBD2173
:1003E000BD1BC4213D080319932108008F08031980
:1003F00008008F0196308E00D00FB02AD00ABD1AA7
:10040000282A521C282A521F192AD41C0A2AD4012D
:100410005415362A541D0F2AD401D415362AD41D5A
:10042000142AD4015416362A541E362AD401D41460
:10043000362A541D1E2AD4015416362AD41D232AC6
:10044000D4015416362A541E362AD401D414362A1E
:10045000D41C2D2AD4015415362A541D322AD40115
:10046000D415362A541E362AD4015415BD1A5F2AD3
:10047000D21C5F2AD21F502AD51C412AD5015515FE
:100480006D2A551D462AD501D5156D2AD51D4B2A35
:10049000D50155166D2A551E6D2AD501D5146D2A24
:1004A000551D552AD50155166D2AD51D5A2AD50137
:1004B00055166D2A551E6D2AD501D5146D2AD51CE9
:1004C000642AD50155156D2A551D692AD501D51502
:1004D0006D2A551E6D2AD5015515531C7E2A561DB1
:1004E000742AD60156168C2AD61D792AD60156169C
:1004F0008C2A561E8C2AD601D6148C2AD61C832A06
:10050000D60156158C2A561D882AD601D6158C2A56
:10051000561E8C2AD6015615D31C9D2A571D932A88
:10052000D7015716AB2AD71D982AD7015716AB2AE1
:10053000571EAB2AD701D714AB2AD71CA22AD70142
:100540005715AB2A571DA72AD701D715AB2A571E17
:10055000AB2AD701571569214E08D2004F08D300A6
:100560005008D1000C305405031D85100C30550582
:10057000031D05100C305605031D85120C30570560
:10058000031D051251080E020318DA2A1230540511
:10059000031D851412305505031D05141230560530
:1005A000031D851612305705031D0516FF30500236
:1005B000031908008F08031D08007B2051080E0254
:1005C000031CDA2A18305405031D85100630540523
:1005D000031D851418305505031D051006305505FB
:1005E000031D051418305605031D851206305605E7
:1005F000031D851618305705031D051206305705D3
:06060000031D05160800B1
:084000000E000300060005009C
:02400E00CC01E3
:10420000010078007A007C007E007B0079007F004E
:104210007D007A0078007E007C00FF00FF00FF0038
:104220000000F200F600FA00FE00F200F600FA00CC
:10423000FE00F200F600FA00FE00FF00FF00FF00A3
:10424000010005000500050005000900090009003E
:1042500009000D000D000D000D00FF00FF00FF0024
:10426000FF00FF00FF00FF00FF00FF00FF00FF0056
:10427000FF00FF00FF00FF00FF00FF00FF00FF0046
:10428000FF00FF00FF00FF00FF00FF00FF00FF0036
:10429000FF00FF00FF00FF00FF00FF00FF00FF0026
:1042A000FF00FF00FF00FF00FF00FF00FF00FF0016
:1042B000FF00FF00FF00FF00FF00FF00FF00FF0006
:1042C000FF00FF00FF00FF00FF00FF00FF00FF00F6
:1042D000FF00FF00FF00FF00FF00FF00FF00FF00E6
:1042E000FF00FF00FF00FF00FF00FF00FF00FF00D6
:1042F000FF00FF00FF00FF00FF00FF00FF00DD00E8
:00000001FF
